:100000000C942A001895000018950000189500001F
:10001000189500001895000018950000189500002C
:10002000189500001895000018950000189500001C
:10003000189500001895000018950000189500000C
:1000400018950000189500001895000018950000FC
:10005000189500008FE58DBFC0E2E8E14E2E88E0E4
:100060008EBFD8E0F7E05F2EA89584B7082E877F73
:1000700084BF88E1992781BD91BDEEEFF7E0A0E64E
:10008000B0E088278D933197E9F76624BA9ABB9A36
:10009000B89AB99A8FEF8ABB8FEF84BBC298C39A84
:1000A000C19A70E07BBB70E075BBBC9AC498BD9AE6
:1000B000C59ABE9AC69ABF9AC79884E08093650095
:1000C00083E08093700080E08093710080E08093F3
:1000D000720080E080937300709174007F7770935A
:1000E000740080E890E0A5E7B0E08D939C9380E8F1
:1000F0008093770080E081BBA9E7B0E00E94772D74
:1001000080E0D2018C9381E00E94552D0E9424272B
:10011000229681E00E94512DD2010E94772D82E02B
:100120000E94552D0E949229229682E00E94512D14
:1001300080E080936400D201E2E6FBE50E94652D39
:100140008AE20E94552DD2010E94772D82E00E9402
:10015000552D84E190E0D2018D939C9382E00E9422
:10016000552D83E0D2018C9381E00E94552D80EEC5
:100170009FEFD2018D939C9382E00E94552DD20176
:100180000E94772D82E00E94552D0E94E3292C9633
:1001900083E30E94512D84EF91E00E943F2DD20114
:1001A000ECE8FBE50E94652D8AE20E94552DD20104
:1001B0000E94772D82E00E94552D84E190E0D201CB
:1001C0008D939C9382E00E94552D83E0D2018C9305
:1001D00081E00E94552DD2010E94772D82E00E947D
:1001E000552DD2010E94772D82E00E94552D0E944C
:1001F000E3292C9683E30E94512D0E949E0980E002
:1002000098EFA0E9B0E08D939C930E9462048CE18A
:1002100096E8A0E9B0E08D939C930E94B802A4E711
:10022000B0E08C9187FBA8E3B0E08C9187F98C93C8
:10023000A5E6B0E08C9180FBA8E3B0E08C9186F954
:100240008C93A5E6B0E08C9181FBA8E3B0E08C91A3
:1002500085F98C93A5E6B0E08C9182FBA8E3B0E031
:100260008C9184F98C930E9497010E94FD030E9457
:10027000F81400917000003011F00C9441010E94BC
:10028000A70B00917000003011F00C9449010E94FE
:10029000A70B00917000013011F00C9451010E94E5
:1002A000A70B81E090E0A6E6B0E08D939C93A6E6D4
:1002B000B0E00D911C91003054E0150718F011F0DA
:1002C0000C948901A6E6B0E0AD90BD90AFEFB0E030
:1002D000AA0DBB1D0C910F3F81E009F080E08F93C8
:1002E00000916500003080E010F009F081E09F91FE
:1002F0008923882311F40C94820180916500815038
:1003000080936500A6E6B0E00E94E82C10F40C94FF
:1003100057010E94760C0E94F50C8FE190E0A0E955
:10032000B0E08D939C930E94B8020C9433018FEF40
:10033000809372007FEF75BB80E084BBA2E7B0E0E2
:1003400083B38C938FEF84BBA2E7B0E00C9103FBE7
:1003500016F40C94BE01A3E7B0E08C918F5F8C93F0
:1003600000917300033018F011F00C94B9010C9453
:10037000BC0180E0809373000E946204A2E7B0E0B9
:100380000C9102FB16F40C94D801809173008150FB
:100390008093730000917300083C18F011F00C94E6
:1003A000D3010C94D60183E0809373000E94620411
:1003B000A2E7B0E00C9101FB81E00EF480E08F93A6
:1003C000A2E7B0E00C9104FB81E00EF480E09F9185
:1003D000892B882311F40C94B7020091730000302C
:1003E00011F00C943B02A2E7B0E00C9101FB16F473
:1003F0000C940102A5E6B0E08C9181508C930C9492
:100400000602A5E6B0E08C918F5F8C9300916500A9
:10041000083C18F011F00C940F020C94120280E0CA
:100420008093650000916500073018F011F00C947E
:100430001B020C941E0287E080936500A5E6B0E0E5
:100440008C9180FBA8E3B0E08C9186F98C93A5E6B3
:10045000B0E08C9181FBA8E3B0E08C9185F98C939E
:10046000A5E6B0E08C9182FBA8E3B0E08C9184F922
:100470008C930E94620400917300013011F00C947F
:100480007002A2E7B0E00C9101FB16F40C944F024D
:10049000A0E7B0E08C918F5F8C930C945402A0E79E
:1004A000B0E08C9181508C9300917000083C18F062
:1004B00011F00C945D020C94600280E08093700057
:1004C00000917000093018F011F00C9469020C943E
:1004D0006C0289E0809370000E949E090E94620471
:1004E00000917300023011F00C948E02A4E7B0E08A
:1004F0008C9187FB882780F9809580FBA4E7B0E08A
:100500008C9187F98C93A4E7B0E08C9187FBA8E3EA
:10051000B0E08C9187F98C930E9462040091730083
:10052000033011F00C94B702A0E9B0E00E94772DDF
:100530000E94B802A2E7B0E00C9101FB16F40C9403
:10054000A802A7E7B0E08C9184508C930C94AD0284
:10055000A7E7B0E08C918C5F8C938CE196E8A0E9E2
:10056000B0E08D939C930E94B8020E9462040895AB
:1005700081E090E0D2018D939C9382E00E94552D02
:10058000A7E7B0E00D911127045F1F4FD2010D9333
:100590001C9382E00E94552DA0E9B0E08D919C91C2
:1005A000D2018D939C9382E00E94552D0E94E62BF0
:1005B000269686E00E94512D81E090E0D2018D9335
:1005C0009C9382E00E94552DA7E7B0E00D91112782
:1005D000055F1F4FD2010D931C9382E00E94552DA1
:1005E000A0E9B0E08D919C91D2018D939C9382E023
:1005F0000E94552D0E94E62B269686E00E94512DE2
:1006000081E090E0D2018D939C9382E00E94552D71
:10061000A7E7B0E00D911127065F1F4FD2010D93A0
:100620001C9382E00E94552DA0E9B0E08D919C9131
:10063000D2018D939C9382E00E94552D0E94E62B5F
:10064000269686E00E94512D81E090E0D2018D93A4
:100650009C9382E00E94552DA7E7B0E00D911127F1
:10066000075F1F4FD2010D931C9382E00E94552D0E
:10067000A0E9B0E08D919C91D2018D939C9382E092
:100680000E94552D0E94E62B269686E00E94512D51
:1006900081E090E0D2018D939C9382E00E94552DE1
:1006A000A7E7B0E00D911127085F1F4FD2010D930E
:1006B0001C9382E00E94552DA0E9B0E08D919C91A1
:1006C000D2018D939C9382E00E94552D0E94E62BCF
:1006D000269686E00E94512D82E090E0D2018D9313
:1006E0009C9382E00E94552DA7E7B0E00D91112761
:1006F000055F1F4FD2010D931C9382E00E94552D80
:10070000A0E9B0E08D919C91D2018D939C9382E001
:100710000E94552D0E94E62B269686E00E94512DC0
:1007200082E090E0D2018D939C9382E00E94552D4F
:10073000A7E7B0E00D911127065F1F4FD2010D937F
:100740001C9382E00E94552DA0E9B0E08D919C9110
:10075000D2018D939C9382E00E94552D0E94E62B3E
:10076000269686E00E94512D82E090E0D2018D9382
:100770009C9382E00E94552DA7E7B0E00D911127D0
:10078000075F1F4FD2010D931C9382E00E94552DED
:10079000A0E9B0E08D919C91D2018D939C9382E071
:1007A0000E94552D0E94E62B269686E00E94512D30
:1007B00083E090E0D2018D939C9382E00E94552DBE
:1007C000A7E7B0E00D911127065F1F4FD2010D93EF
:1007D0001C9382E00E94552DA0E9B0E08D919C9180
:1007E000D2018D939C9382E00E94552D0E94E62BAE
:1007F000269686E00E94512D08958FE190E0A0E9B1
:10080000B0E08D939C93A6E6B0E00E94772DA6E61B
:10081000B0E00D911C910F3D51E0150718F011F05B
:100820000C9461048AE090E0A8E6B0E08D939C937C
:10083000A8E6B0E00D911C91093051E0150718F0C1
:1008400011F00C945404A6E6B0E08D919C91D20175
:100850008D939C9382E00E94552DA8E6B0E08D9187
:100860009C91D2018D939C9382E00E94552DA0E92A
:10087000B0E08D919C91D2018D939C9382E00E9477
:10088000552D0E94E62B269686E00E94512DA8E663
:10089000B0E00D911C910C5E1F4FA8E6B0E00D93E7
:1008A0001C9310F40C941804A6E6B0E00D911C9172
:1008B000085D1F4FA6E6B0E00D931C9310F40C9456
:1008C00007040895A6E6B0E00E94772DA6E6B0E002
:1008D0000D911C914CE050E00E945B2DA8E6B0E029
:1008E0000D931C9380EE9FEFA0E9B0E08D939C9355
:1008F00000916500003011F00C948404AFE7B0E083
:10090000E6EBFBE50E94652D00916500013011F0DA
:100910000C949004AFE7B0E0ECEBFBE50E94652D92
:1009200000916500023011F00C949C04AFE7B0E038
:10093000E2ECFBE50E94652D00916500033011F0AB
:100940000C94A804AFE7B0E0E8ECFBE50E94652D4D
:1009500000916500043011F00C94B404AFE7B0E0EE
:10096000EEECFBE50E94652D00916500053011F06D
:100970000C94C004AFE7B0E0E4EDFBE50E94652D08
:1009800000916500063011F00C94CC04AFE7B0E0A4
:10099000EAEDFBE50E94652D00916500073011F03E
:1009A0000C94D804AFE7B0E0E0EEFBE50E94652DC3
:1009B00000917300003011F00C941805EFE7F0E09F
:1009C000D2010E94872D8FE00E94552DA8E6B0E04D
:1009D0008D919C91D2018D939C9382E00E94552D24
:1009E00088E191E0D2018D939C9382E00E94552D85
:1009F00083E0D2018C9381E00E94552D8CE196E832
:100A0000D2018D939C9382E00E94552DA0E9B0E025
:100A10008D919C91D2018D939C9382E00E94552DE3
:100A20000E94E3292C9688E10E94512D0C944C05DC
:100A3000EFE7F0E0D2010E94872D8FE00E94552D54
:100A4000A8E6B0E08D919C91D2018D939C9382E0B9
:100A50000E94552D88E191E0D2018D939C9382E014
:100A60000E94552D83E0D2018C9381E00E94552D88
:100A70008CE196E8D2018D939C9382E00E94552DE3
:100A8000D2010E94772D82E00E94552D0E94E32919
:100A90002C9688E10E94512D85E090E0A6E6B0E01A
:100AA0008D939C93A6E6B0E00D911C914CE050E034
:100AB0000E945B2DA8E6B0E00D931C93D201E6EEF8
:100AC000FBE50E94652D82E00E94552DA8E6B0E06E
:100AD0008D919C91D2018D939C9382E00E94552D23
:100AE00088E191E0D2018D939C9382E00E94552D84
:100AF00083E0D2018C9381E00E94552D8CE196E831
:100B0000D2018D939C9382E00E94552DD2010E94C8
:100B1000772D82E00E94552D0E94E3292C968BE0D0
:100B20000E94512D86E090E0A6E6B0E08D939C9364
:100B3000A6E6B0E00D911C914CE050E00E945B2DC8
:100B4000A8E6B0E00D931C9300917000003011F006
:100B50000C94B005AFE7B0E0E8EEFBE50E94652D30
:100B600000917000013011F00C94BC05AFE7B0E0CB
:100B7000E0EFFBE50E94652D00917000023011F05E
:100B80000C94C805AFE7B0E0E8EFFBE50E94652DE7
:100B900000917000033011F00C94D405AFE7B0E081
:100BA000E0E0FCE50E94652D00917000043011F03A
:100BB0000C94E005AFE7B0E0E8E0FCE50E94652DAD
:100BC00000917000053011F00C94EC05AFE7B0E037
:100BD000E0E1FCE50E94652D00917000063011F007
:100BE0000C94F805AFE7B0E0E8E1FCE50E94652D64
:100BF00000917000073011F00C940406AFE7B0E0EC
:100C0000E0E2FCE50E94652D00917000083011F0D3
:100C10000C941006AFE7B0E0E8E2FCE50E94652D19
:100C200000917000093011F00C941C06AFE7B0E0A1
:100C3000E0E3FCE50E94652D00917100013011F0A8
:100C40000C942806AFE7B0E0E8E3FCE50E94652DD0
:100C500000917300013011F00C946806EFE7F0E0AA
:100C6000D2010E94872D8FE00E94552DA8E6B0E0AA
:100C70008D919C91D2018D939C9382E00E94552D81
:100C800088E191E0D2018D939C9382E00E94552DE2
:100C900083E0D2018C9381E00E94552D8CE196E88F
:100CA000D2018D939C9382E00E94552DA0E9B0E083
:100CB0008D919C91D2018D939C9382E00E94552D41
:100CC0000E94E3292C9688E10E94512D0C949C06E9
:100CD000EFE7F0E0D2010E94872D8FE00E94552DB2
:100CE000A8E6B0E08D919C91D2018D939C9382E017
:100CF0000E94552D88E191E0D2018D939C9382E072
:100D00000E94552D83E0D2018C9381E00E94552DE5
:100D10008CE196E8D2018D939C9382E00E94552D40
:100D2000D2010E94772D82E00E94552D0E94E32976
:100D30002C9688E10E94512D8DE090E0A6E6B0E06F
:100D40008D939C93A6E6B0E00D911C914CE050E091
:100D50000E945B2DA8E6B0E00D931C93D201E6EE55
:100D6000FBE50E94652D82E00E94552DA8E6B0E0CB
:100D70008D919C91D2018D939C9382E00E94552D80
:100D800088E191E0D2018D939C9382E00E94552DE1
:100D900083E0D2018C9381E00E94552D8CE196E88E
:100DA000D2018D939C9382E00E94552DD2010E9426
:100DB000772D82E00E94552D0E94E3292C968BE02E
:100DC0000E94512D8EE090E0A6E6B0E08D939C93BA
:100DD000A6E6B0E00D911C914CE050E00E945B2D26
:100DE000A8E6B0E00D931C93A4E7B0E08C9187FBDC
:100DF00016F40C940107AFE7B0E0E2E4FCE50E94D2
:100E0000652DA4E7B0E08C9187FB16F00C940E07DB
:100E1000AFE7B0E0E6E4FCE50E94652D00917300C9
:100E2000023011F00C944E07EFE7F0E0D2010E947F
:100E3000872D8FE00E94552DA8E6B0E08D919C9102
:100E4000D2018D939C9382E00E94552D88E191E020
:100E5000D2018D939C9382E00E94552D83E0D201B4
:100E60008C9381E00E94552D8CE196E8D2018D9300
:100E70009C9382E00E94552DA0E9B0E08D919C9159
:100E8000D2018D939C9382E00E94552D0E94E3290C
:100E90002C9688E10E94512D0C948207EFE7F0E038
:100EA000D2010E94872D8FE00E94552DA8E6B0E068
:100EB0008D919C91D2018D939C9382E00E94552D3F
:100EC00088E191E0D2018D939C9382E00E94552DA0
:100ED00083E0D2018C9381E00E94552D8CE196E84D
:100EE000D2018D939C9382E00E94552DD2010E94E5
:100EF000772D82E00E94552D0E94E3292C9688E1EF
:100F00000E94512D81E190E0A6E6B0E08D939C9384
:100F1000A6E6B0E00D911C914CE050E00E945B2DE4
:100F2000A8E6B0E00D931C93D201EAE4FCE50E9430
:100F3000652D83E00E94552DA8E6B0E08D919C912F
:100F4000D2018D939C9382E00E94552D88E191E01F
:100F5000D2018D939C9382E00E94552D83E0D201B3
:100F60008C9381E00E94552D8CE196E8D2018D93FF
:100F70009C9382E00E94552DD2010E94772D82E041
:100F80000E94552D0E94E3292C968CE00E94512D41
:100F900083E190E0A6E6B0E08D939C93A6E6B0E0F6
:100FA0000D911C914CE050E00E945B2DA8E6B0E052
:100FB0000D931C9300917300033011F00C941A08E8
:100FC000D201EEE4FCE50E94652D85E00E94552DDE
:100FD000A8E6B0E08D919C91D2018D939C9382E024
:100FE0000E94552D88E191E0D2018D939C9382E07F
:100FF0000E94552D83E0D2018C9381E00E94552DF3
:101000008CE196E8D2018D939C9382E00E94552D4D
:10101000A0E9B0E08D919C91D2018D939C9382E0E8
:101020000E94552D0E94E3292C968EE00E94512D9E
:101030000C944E08D201EEE4FCE50E94652D85E09B
:101040000E94552DA8E6B0E08D919C91D2018D9320
:101050009C9382E00E94552D88E191E0D2018D930E
:101060009C9382E00E94552D83E0D2018C9381E015
:101070000E94552D8CE196E8D2018D939C9382E0DD
:101080000E94552DD2010E94772D82E00E94552D9D
:101090000E94E3292C968EE00E94512D87E190E07A
:1010A000A6E6B0E08D939C93A6E6B0E00D911C916E
:1010B0004CE050E00E945B2DA8E6B0E00D931C933D
:1010C000D201E6EEFBE50E94652D82E00E94552DDF
:1010D000A8E6B0E08D919C91D2018D939C9382E023
:1010E0000E94552D88E191E0D2018D939C9382E07E
:1010F0000E94552D83E0D2018C9381E00E94552DF2
:101100008CE196E8D2018D939C9382E00E94552D4C
:10111000D2010E94772D82E00E94552D0E94E32982
:101120002C968BE00E94512DA6E6B0E00E94772D10
:10113000A8E6B0E00E94772D80E0809364000895D7
:1011400080E080936400D201E4E5FCE50E94652D17
:1011500086E00E94552D82E090E0D2018D939C9311
:1011600082E00E94552D88E090E0D2018D939C93FF
:1011700082E00E94552D81E0D2018C9381E00E9493
:10118000552D80EE9FEFD2018D939C9382E00E94BB
:10119000552DD2010E94772D82E00E94552D0E948C
:1011A000E3292C968FE00E94512DD201EAE5FCE55F
:1011B0000E94652D86E00E94552D82E090E0D201CC
:1011C0008D939C9382E00E94552D88E490E0D2019B
:1011D0008D939C9382E00E94552D81E0D2018C93E7
:1011E00081E00E94552D80EE9FEFD2018D939C935C
:1011F00082E00E94552DD2010E94772D82E00E944C
:10120000552D0E94E3292C968FE00E94512DD2018A
:10121000E0E6FCE50E94652D86E00E94552D82E007
:1012200090E0D2018D939C9382E00E94552D88E836
:1012300090E0D2018D939C9382E00E94552D81E035
:10124000D2018C9381E00E94552D80EE9FEFD20158
:101250008D939C9382E00E94552DD2010E94772DA0
:1012600082E00E94552D0E94E3292C968FE00E9477
:10127000512DD201E6E6FCE50E94652D86E00E9434
:10128000552D82E090E0D2018D939C9382E00E94E4
:10129000552D88EC90E0D2018D939C9382E00E94C2
:1012A000552D81E0D2018C9381E00E94552D80EE76
:1012B0009FEFD2018D939C9382E00E94552DD20125
:1012C0000E94772D82E00E94552D0E94E3292C96E2
:1012D0008FE00E94512DD201ECE6FCE50E94652DC5
:1012E00086E00E94552D82E090E0D2018D939C9380
:1012F00082E00E94552D84E091E0D2018D939C9371
:1013000082E00E94552D81E0D2018C9381E00E9401
:10131000552D80EE9FEFD2018D939C9382E00E9429
:10132000552DD2010E94772D82E00E94552D0E94FA
:10133000E3292C968FE00E94512D089500917000B2
:10134000003011F00C94D209D201E2E7FCE50E94D2
:10135000652D8BE30E94552DD2010E94772D82E0EE
:101360000E94552DD2010E94772D82E00E94552DBA
:1013700081E0D2018C9381E00E94552D8CE196E8AA
:10138000D2018D939C9382E00E94552DD2010E9440
:10139000772D82E00E94552D0E94E3292C9684E44B
:1013A0000E94512D00917000013011F00C94060A3A
:1013B000D201EEEAFCE50E94652D8CE30E94552DDA
:1013C000D2010E94772D82E00E94552DD2010E9409
:1013D000772D82E00E94552D81E0D2018C9381E02F
:1013E0000E94552D8CE196E8D2018D939C9382E06A
:1013F0000E94552DD2010E94772D82E00E94552D2A
:101400000E94E3292C9685E40E94512D00917000E2
:10141000023011F00C943A0AD201EAEEFCE50E9487
:10142000652D8BE30E94552DD2010E94772D82E01D
:101430000E94552DD2010E94772D82E00E94552DE9
:1014400081E0D2018C9381E00E94552D8CE196E8D9
:10145000D2018D939C9382E00E94552DD2010E946F
:10146000772D82E00E94552D0E94E3292C9684E47A
:101470000E94512D00917000033011F00C946E0AFF
:10148000D201E6E2FDE50E94652D8BE30E94552D19
:10149000D2010E94772D82E00E94552DD2010E9438
:1014A000772D82E00E94552D81E0D2018C9381E05E
:1014B0000E94552D8CE196E8D2018D939C9382E099
:1014C0000E94552DD2010E94772D82E00E94552D59
:1014D0000E94E3292C9684E40E94512D0091700013
:1014E000043011F00C94A20AD201E2E6FDE50E945C
:1014F000652D8BE30E94552DD2010E94772D82E04D
:101500000E94552DD2010E94772D82E00E94552D18
:1015100081E0D2018C9381E00E94552D8CE196E808
:10152000D2018D939C9382E00E94552DD2010E949E
:10153000772D82E00E94552D0E94E3292C9684E4A9
:101540000E94512D00917000053011F00C94D60AC4
:10155000D201EEE9FDE50E94652D8BE30E94552D39
:10156000D2010E94772D82E00E94552DD2010E9467
:10157000772D82E00E94552D81E0D2018C9381E08D
:101580000E94552D8CE196E8D2018D939C9382E0C8
:101590000E94552DD2010E94772D82E00E94552D88
:1015A0000E94E3292C9684E40E94512D0091700042
:1015B000063011F00C940A0BD201EAEDFDE50E9411
:1015C000652D8BE30E94552DD2010E94772D82E07C
:1015D0000E94552DD2010E94772D82E00E94552D48
:1015E00081E0D2018C9381E00E94552D8CE196E838
:1015F000D2018D939C9382E00E94552DD2010E94CE
:10160000772D82E00E94552D0E94E3292C9684E4D8
:101610000E94512D00917000073011F00C943E0B88
:10162000D201E6E1FEE50E94652D8BE30E94552D77
:10163000D2010E94772D82E00E94552DD2010E9496
:10164000772D82E00E94552D81E0D2018C9381E0BC
:101650000E94552D8CE196E8D2018D939C9382E0F7
:101660000E94552DD2010E94772D82E00E94552DB7
:101670000E94E3292C9684E40E94512D0091700071
:10168000083011F00C94720BD201E2E5FEE50E94E5
:10169000652D8BE30E94552DD2010E94772D82E0AB
:1016A0000E94552DD2010E94772D82E00E94552D77
:1016B00081E0D2018C9381E00E94552D8CE196E867
:1016C000D2018D939C9382E00E94552DD2010E94FD
:1016D000772D82E00E94552D0E94E3292C9684E408
:1016E0000E94512D00917000093011F00C94A60B4E
:1016F000D201EEE8FEE50E94652D8BE30E94552D98
:10170000D2010E94772D82E00E94552DD2010E94C5
:10171000772D82E00E94552D81E0D2018C9381E0EB
:101720000E94552D8CE196E8D2018D939C9382E026
:101730000E94552DD2010E94772D82E00E94552DE6
:101740000E94E3292C9684E40E94512D089580E0A4
:1017500094E0A6E6B0E08D939C93A6E6B0E04D91B0
:101760005C9101E010E00417150718F011F00C94DB
:10177000EC0BA6E6B0E00D911C9142E050E00E9417
:101780001C2DA8E6B0E04D935C93A8E6B0E0AD90C8
:10179000BD90AFEFB0E0AA0DBB1D8C91A6E6B0E006
:1017A000AD90BD90AFEFB0E0AA0DBB1D8C93A6E647
:1017B000B0E0AD90BD90AFEFB0E0AA0DBB1D8C9135
:1017C000AAE6B0E08D9388278C93A6E6B0E00E944D
:1017D000EF2C10F00C94AD0B82E090E0A6E6B0E0A8
:1017E0008D939C93A6E6B0E00D911C910F3F53E0C2
:1017F000150718F011F00C943D0CA6E6B0E0AD9082
:10180000BD90AEEFB0E0AA0DBB1D0D911127A6E66D
:10181000B0E0AD90BD90A0E0B1E0AA0DBB1D4D9130
:101820005527040F151FAAE6B0E00D931C93AAE6F6
:10183000B0E00D911C9142E050E00E941C2DAAE600
:10184000B0E04D935C9300916A0041E0049FA6E6EE
:10185000B0E0AD90BD90AFEFB0E0AA0DBB1D0C9213
:10186000A6E6B0E00D911C910E5F1F4FA6E6B0E01A
:101870000D931C9310F40C94F20B089580E094E007
:10188000A6E6B0E08D939C93A6E6B0E04D915C9106
:1018900001E010E00417150718F011F00C94750C16
:1018A000A6E6B0E00D911C9144E050E00E941C2D92
:1018B000A8E6B0E04D935C93A8E6B0E0AD90BD9093
:1018C000AFEFB0E0AA0DBB1D8C91A6E6B0E0AD90E5
:1018D000BD90AFEFB0E0AA0DBB1D8C93A6E6B0E0C3
:1018E0000E94EF2C10F00C94440C0895A8E6B0E090
:1018F0000E94772DAAE6B0E00E94772D83E090E069
:10190000A6E6B0E08D939C93A6E6B0E00D911C9105
:10191000003052E0150718F011F00C94EE0C4091D5
:101920007700A6E6B0E0AD90BD90AFEFB0E0AA0DB5
:10193000BB1D0C91041781E008F080E08F93AAE6AC
:10194000B0E00D911C91003050E0150781E009F0E6
:1019500080E09F918923882311F40C94B50C81E0D9
:1019600090E0A8E6B0E08D939C9340917700A6E6C6
:10197000B0E0AD90BD90AFEFB0E0AA0DBB1D0C91F3
:10198000041781E008F480E08F93A8E6B0E00D91A1
:101990001C91013050E0150781E009F080E09F9133
:1019A0008923882311F40C94E70C81E090E0AAE6E7
:1019B000B0E08D939C93A6E6B0E00D911C9102508F
:1019C0001040A5E7B0E00D931C930C94F40CA6E630
:1019D000B0E00E94E82C10F40C94840C80E092E0BB
:1019E000A5E7B0E08D939C93089581E090E0A6E692
:1019F000B0E08D939C93A6E6B0E00D911C91003E63
:101A000051E0150718F011F00C94B50EA6E6B0E001
:101A10000D911C9101501040AEE8B0E00D931C9365
:101A2000A6E6B0E0AD90BD90A0E0B5E0AA0DBB1D6C
:101A30004C91A6E6B0E0AD90BD90AFEFB4E0AA0D3A
:101A4000BB1D0C91041710F00C94810D81E00E94D5
:101A5000552DA6E6B0E0AD90BD90A0E0B5E0AA0D92
:101A6000BB1D8C91A881B9818C93A6E6B0E0AD90A6
:101A7000BD90AFEFB4E0AA0DBB1D8C91A8E6B0E01D
:101A80008D9388278C93A881B9814D915527A8E61D
:101A9000B0E00D911C910417150718F011F00C948B
:101AA0007A0DAEE8B0E08D919C91D2018D939C931C
:101AB00082E00E94552DA8E6B0E00D911C91065FD2
:101AC0001F4FD2010D931C9382E00E94552DD2012D
:101AD0000E94772D82E00E94552D0E94E62B2696CB
:101AE00086E00E94512DA8E6B0E00E94E82C10F498
:101AF0000C94430D81E0481A80E0580A22960C9419
:101B0000CC0DA6E6B0E0AD90BD90A0E0B5E0AA0D8A
:101B1000BB1D8C91A8E6B0E08D9388278C93A6E638
:101B2000B0E0AD90BD90AFEFB4E0AA0DBB1D4D91FC
:101B30005527A8E6B0E00D911C910417150718F081
:101B400011F00C94CC0DAEE8B0E08D919C91D201D7
:101B50008D939C9382E00E94552DA8E6B0E00D91F4
:101B60001C91065F1F4FD2010D931C9382E00E94CF
:101B7000552DD2010E94772D82E00E94552D0E94A2
:101B8000E62B269686E00E94512DA8E6B0E00E9442
:101B9000E82C10F40C948F0DA6E6B0E00D911C918A
:101BA000A5E7B0E04D915C91040F151FACE6B0E0E5
:101BB0000D931C93ACE6B0E0AD90BD90A0E0B1E019
:101BC000AA0DBB1D4C91ACE6B0E0AD90BD90AFEF5F
:101BD000B0E0AA0DBB1D0C91041710F00C94570E29
:101BE00081E00E94552DACE6B0E0AD90BD90A0E044
:101BF000B1E0AA0DBB1D8C91A881B9818C93ACE694
:101C0000B0E0AD90BD90AFEFB0E0AA0DBB1D8C91E0
:101C1000A8E6B0E08D9388278C93A881B9814D9177
:101C20005527A8E6B0E00D911C910417150718F090
:101C300011F00C94500EACE6B0E00D911C91013007
:101C400054E0150710F00C94490EAEE8B0E08D9109
:101C50009C91D2018D939C9382E00E94552DA8E621
:101C6000B0E00D911C91065F1F4FD2010D931C93A4
:101C700082E00E94552D80E098EFD2018D939C93D5
:101C800082E00E94552D0E94E62B269686E00E9457
:101C9000512DA8E6B0E00E94E82C10F40C940D0E33
:101CA00081E0481A80E0580A22960C94AE0EACE609
:101CB000B0E0AD90BD90A0E0B1E0AA0DBB1D8C914D
:101CC000A8E6B0E08D9388278C93ACE6B0E0AD90A9
:101CD000BD90AFEFB0E0AA0DBB1D4D915527A8E612
:101CE000B0E00D911C910417150718F011F00C9439
:101CF000AE0EACE6B0E00D911C91013054E015073A
:101D000010F00C94A70EAEE8B0E08D919C91D2013A
:101D10008D939C9382E00E94552DA8E6B0E00D9132
:101D20001C91065F1F4FD2010D931C9382E00E940D
:101D3000552D80E098EFD2018D939C9382E00E9414
:101D4000552D0E94E62B269686E00E94512DA8E68E
:101D5000B0E00E94E82C10F40C94650EA6E6B0E00A
:101D60000E94E82C10F40C94FB0C81E090E0A6E6B5
:101D7000B0E08D939C93A6E6B0E00D911C91003EDF
:101D800051E0150718F011F00C94FB0EA6E6B0E038
:101D90000D911C91A5E7B0E04D915C91040F151FCA
:101DA000ACE6B0E00D931C93ACE6B0E00D911C9155
:101DB000A9E7B0E04D915C91040F151FACE6B0E0CF
:101DC0000D931C93ACE6B0E0AD90BD90AFEFB0E0EA
:101DD000AA0DBB1D8C91A6E6B0E0AD90BD90AFEF13
:101DE000B4E0AA0DBB1D8C93A6E6B0E00E94E82CDF
:101DF00010F40C94BB0E08950108080000000000C8
:101E0000000000000000065F06000000000703005D
:101E10000703000000247E247E24000000242B6A97
:101E20001200000000631308646300000036495686
:101E300020500000000007030000000000003E41A9
:101E4000000000000000413E0000000000083E1CB1
:101E50003E0800000008083E080800000000E0609E
:101E6000000000000008080808080000000060608A
:101E7000000000000020100804020000003E51494C
:101E8000453E00000000427F4000000000625149D2
:101E90004946000000224949493600000018141242
:101EA0007F100000002F494949310000003C4A4999
:101EB000493000000001710905030000003649495E
:101EC0004936000000064949291E000000006C6CDC
:101ED000000000000000EC6C00000000000814226C
:101EE000410000000024242424240000000041229A
:101EF000140800000002015909060000003E415D7F
:101F0000551E0000007E1111117E0000007F49491E
:101F100049360000003E414141220000007F41411E
:101F2000413E0000007F494949410000007F090906
:101F300009010000003E4149497A0000007F08087D
:101F4000087F00000000417F410000000030404059
:101F5000403F0000007F081422410000007F404005
:101F600040400000007F0204027F0000007F020466
:101F7000087F0000003E4141413E0000007F09090A
:101F800009060000003E4151215E0000007F090962
:101F90001966000000264949493200000001017F0E
:101FA00001010000003F4040403F0000001F204072
:101FB000201F0000003F403C403F00000063140829
:101FC000146300000007087008070000007149450D
:101FD0004300000000007F414100000000020408AF
:101FE00010200000000041417F00000000040201B9
:101FF00002040000808080808080808000000307D1
:10200000000000000020545454780000007F444435
:102010004438000000384444442800000038444458
:10202000447F0000003854545408000000087E0922
:10203000090000000018A4A4A47C0000007F040490
:10204000780000000000007D400000000040808417
:102050007D000000007F1028440000000000007F89
:1020600040000000007C041804780000007C040498
:1020700078000000003844444438000000FC444428
:10208000443800000038444444FC000000447844D4
:1020900004080000000854545420000000043E448A
:1020A00024000000003C40207C000000001C204078
:1020B000201C0000003C6030603C0000006C1010F0
:1020C0006C000000009CA0603C00000000645454C0
:1020D0004C00000000083E41410000000000007775
:1020E00000000000000041413E080000020C180200
:1020F00000000000000000000000000000000000E0
:102100000000000000000000000000007CFFFF7CD9
:102110000000000000000000003333000000000059
:102120000000263E1E0000263E1E000000000000AB
:10213000000000000000000000000010F0FE1E1073
:10214000F0FE1E100000021E1F03021E1F030000EF
:10215000000078FCCCFFFFCCCC8800000000040C11
:102160000C3F3F0C0F0700000000386C6C3880C03B
:10217000E070381C0000181C0E0703011C36361CCA
:10218000000000B8FCC6E23E1C00000000001F3F3B
:102190003121371E1C36220000000000263E1E00A2
:1021A000000000000000000000000000000000002F
:1021B000000000F0FCFE0701010000000000000329
:1021C0000F1F382020000000000000010107FEFC66
:1021D000F00000000000002020381F0F0300000066
:1021E00000000098B8E0F8F8E0B898000000000C93
:1021F0000E030F0F030E0C00000000808080F0F033
:10220000808080000000000101010F0F010101002A
:1022100000000000000000000000000000000000BE
:10222000004C7C3C0000000000000080808080802A
:102230008080800000000001010101010101010016
:10224000000000000000000000000000000000008E
:102250000038383800000000000000000080C0E0B6
:1022600070381C0E00001C0E070301000000000067
:102270000000F8FE0683C363331EFEF80000071F4C
:102280001B31303030181F070000000C0C0EFFFF10
:10229000000000000000003030303F3F30303000A0
:1022A00000001C1E070383C3E3773E1C0000383C7C
:1022B0003E3733313030303000000C0E07C3C3C31B
:1022C000C3E77E3C00000C1C3830303030391F0E24
:1022D0000000C0E070381C0EFFFF00000000070780
:1022E000060606063F3F06060000787F67636363C5
:1022F00063E3C38300000C1C3830303030381F0FCC
:102300000000C0F0F8DCCEC7C3C3800000000F1F80
:102310003930303030391F0F00000303030303C38B
:10232000F33F0F0300000000303C0F0300000000EB
:10233000000000BCFEE7C3C3E7FEBC0000000F1FA7
:102340003930303030391F0F00003C7EE7C3C3C343
:10235000C3E7FEFC000000303030381C0E070300DD
:10236000000000000070707000000000000000001D
:10237000001C1C1C000000000000000000707070B9
:102380000000000000000000004C7C7C0000000009
:10239000000000C0E0F0381C0E0703000000000041
:1023A0000103070E1C3830000000006060606060B0
:1023B00060606000000000060606060606060600CD
:1023C00000000003070E1C38F0E0C00000000030E1
:1023D000381C0E070301000000001C1E070383C306
:1023E000E3773E1C000000000000373700000000CB
:1023F0000000FCFE03F31BFBFB07FEF800000F1FB1
:10240000303336373736030100000000E0FC1F1F71
:10241000FCE000000000383F0706060606073F38CC
:102420000000FFFFC3C3C3C3E7FEBC0000003F3F83
:102430003030303030391F0F0000F0FC0E0703033E
:1024400003070E0C0000030F1C38303030381C0C12
:102450000000FFFF03030303070EFCF000003F3FF3
:1024600030303030381C0F030000FFFFC3C3C3C33C
:10247000C3C3030300003F3F3030303030303030D2
:102480000000FFFFC3C3C3C3C3C3030300003F3F38
:1024900000000000000000000000F0FC0E0703C375
:1024A000C3C3C7C60000030F1C38303030303F3F75
:1024B0000000FFFFC0C0C0C0C0C0FFFF00003F3F22
:1024C0000000000000003F3F000000000303FFFF8A
:1024D000030300000000000030303F3F30300000B8
:1024E00000000000000000000000FFFF00000E1EC2
:1024F0003830303030381F070000FFFFC0E0F038C0
:102500001C0E070300003F3F000103070E1C38307C
:102510000000FFFF000000000000000000003F3F3F
:1025200030303030303030300000FFFF1E78E0E0D7
:10253000781EFFFF00003F3F0000010100003F3F09
:102540000000FFFF0E38F0C00000FFFF00003F3F1B
:1025500000000003071C3F3F0000F0FC0E070303D0
:10256000070EFCF00000030F1C383030381C0F033E
:102570000000FFFF8383838383C7FE7C00003F3F0F
:1025800001010101010100000000F0FC0E0703033E
:10259000070EFCF00000030F1C3830363E1C3F33A2
:1025A0000000FFFF8383838383C7FE7C00003F3FDF
:1025B000010103070F1D383000003C7EE7C3C3C391
:1025C000C3C78E0C00000C1C3830303030391F0F60
:1025D000000003030303FFFF0303030300000000E5
:1025E00000003F3F000000000000FFFF000000006F
:1025F0000000FFFF0000071F3830303030381F0761
:102600000000073FF8C00000C0F83F0700000000CE
:10261000010F3E3E0F0100000000FFFF0000808020
:102620000000FFFF00003F3F1C060303061C3F3F66
:102630000000030F1C30E0E0301C0F030000303CB2
:102640000E030101030E3C300000030F3CF0C0C03C
:10265000F03C0F030000000000003F3F00000000BE
:10266000000003030303C3E3331F0F030000303CE8
:102670003E3331303030303000000000FFFF0303C4
:1026800003030000000000003F3F30303030000006
:1026900000001C3870E0C080000000000000000056
:1026A00000000103070E1C180000000003030303D1
:1026B000FFFF000000000000303030303F3F0000DE
:1026C000000070381C0E070E1C387000000000005F
:1026D00000000000000000000000000000000000FA
:1026E00000000000C0C0C0C0C0C0C0C0C0C0C0C0EA
:1026F00000000000003E7E460000000000000000D8
:102700000000000000000000000000406060606009
:102710006060E0C000001C3E3333333333333F3F4F
:102720000000FFFFC060606060E0C08000003F3FCD
:102730003030303030381F0F000080C0E060606003
:102740006060C08000000F1F383030303030180813
:10275000000080C0E0606060E0C0FFFF00000F1F6D
:102760003830303030303F3F000080C0E060606083
:102770006060C08000000F1F3B33333333331301DD
:102780000000000000F0F81C0C0C0000000000032A
:10279000037F7F03030300000000C0E0703030308F
:1027A0003030F0F0000001636766666666733F1FB5
:1027B0000000FFFFC0606060E0C0800000003F3F9D
:1027C00000000000003F3F00000000000060ECEC53
:1027D000000000000000000030303F3F30300000BB
:1027E0000000000000000060ECEC000000000000B1
:1027F000307060607F3F0000000000FFFF0080C07D
:10280000E06000000000003F3F03070F1C3830006D
:10281000000000000003FFFF0000000000000000B7
:1028200030303F3F303000000000E0C0E0E0C0C08A
:10283000E0E0C08000003F3F00003F3F00003F3F1E
:10284000000000E0E0C0606060E0C0800000003F89
:102850003F00000000003F3F000080C0E06060607B
:1028600060E0C08000000F1F3830303030381F0F5C
:102870000000F0F0303030303070E0C000007F7F7A
:10288000060C0C0C0C0E07030000C0E0703030305A
:102890003030F0F0000003070E0C0C0C0C067F7FAC
:1028A000000000E0E0C060606060E0C00000003F49
:1028B0003F00000000000000000000C0E060606019
:1028C000606040000000001133333333333F1E009B
:1028D0000000006060FEFE6060600000000000001C
:1028E000001F3F30303030000000E0E0000000000A
:1028F0000000E0E000000F1F3830303030183F3F5C
:10290000000060E0800000000080E0600000000146
:10291000071E38381E0701000000E0E00000E0E07C
:102920000000E0E00000071F381C0F0F1C381F07D5
:10293000000060E0C0800080C0E06000000030382F
:102940001D0F070F1D3830000000000030F0C000E0
:1029500000C0F030000000000040733F0F03000093
:1029600000004060606060E0E060200000003038FF
:102970003C3633313030100000000080C0F87C0E4F
:102980000606060000000000010F1F38303030003E
:10299000000000000000FFFF000000000000000039
:1029A00000003F3F000000000000000606060E7C0D
:1029B000F8C08000000000303030381F0F010000E8
:1029C0000000406030103060406030100000080CA3
:1029D0000602060C080C060200000080C0603030C1
:1029E00060C0800000000F0F0C0C0C0C0C0C0F0FC3
:1029F000A6E6B0E00E94772D00917000003011F043
:102A00000C9404150E947D1500917000013011F0A6
:102A10000C940C150E947D1500917000023011F08D
:102A20000C9414150E947D1500917000033011F074
:102A30000C941C150E949A2500917000043011F02E
:102A40000C9424150E94CE2500917000053011F0E1
:102A50000C942C150E940E2600917000063011F087
:102A60000C9434150E94442600917000073011F038
:102A70000C943C150E947B2600917000083011F0E8
:102A80000C9444150E94B22600917000093011F098
:102A90000C944C150E94E82608954091770000B3ED
:102AA000041718F011F00C9457150C947215A6E643
:102AB000B0E00D911C910F5F1F4FA6E6B0E00D93A3
:102AC0001C93A6E6B0E00D911C91083E53E015075B
:102AD00018F011F00C946E150C9470150C9472157E
:102AE0000C944D15AF93BF93B1E0A0E080B38D93EC
:102AF000B530E0F3BF91AF9108954091770000B3F6
:102B0000041718F011F00C9487150C94A215A6E682
:102B1000B0E00D911C910F5F1F4FA6E6B0E00D9342
:102B20001C93A6E6B0E00D911C91083E53E01507FA
:102B300018F011F00C949E150C94A0150C94A2158D
:102B40000C947D1500B300000093000100B3000059
:102B50000093010100B300000093020100B30000E4
:102B60000093030100B300000093040100B30000D0
:102B70000093050100B300000093060100B30000BC
:102B80000093070100B300000093080100B30000A8
:102B90000093090100B3000000930A0100B3000094
:102BA00000930B0100B3000000930C0100B3000080
:102BB00000930D0100B3000000930E0100B300006C
:102BC00000930F0100B300000093100100B3000058
:102BD0000093110100B300000093120100B3000044
:102BE0000093130100B300000093140100B3000030
:102BF0000093150100B300000093160100B300001C
:102C00000093170100B300000093180100B3000007
:102C10000093190100B3000000931A0100B30000F3
:102C200000931B0100B3000000931C0100B30000DF
:102C300000931D0100B3000000931E0100B30000CB
:102C400000931F0100B300000093200100B30000B7
:102C50000093210100B300000093220100B30000A3
:102C60000093230100B300000093240100B300008F
:102C70000093250100B300000093260100B300007B
:102C80000093270100B300000093280100B3000067
:102C90000093290100B3000000932A0100B3000053
:102CA00000932B0100B3000000932C0100B300003F
:102CB00000932D0100B3000000932E0100B300002B
:102CC00000932F0100B300000093300100B3000017
:102CD0000093310100B300000093320100B3000003
:102CE0000093330100B300000093340100B30000EF
:102CF0000093350100B300000093360100B30000DB
:102D00000093370100B300000093380100B30000C6
:102D10000093390100B3000000933A0100B30000B2
:102D200000933B0100B3000000933C0100B300009E
:102D300000933D0100B3000000933E0100B300008A
:102D400000933F0100B300000093400100B3000076
:102D50000093410100B300000093420100B3000062
:102D60000093430100B300000093440100B300004E
:102D70000093450100B300000093460100B300003A
:102D80000093470100B300000093480100B3000026
:102D90000093490100B3000000934A0100B3000012
:102DA00000934B0100B3000000934C0100B30000FE
:102DB00000934D0100B3000000934E0100B30000EA
:102DC00000934F0100B300000093500100B30000D6
:102DD0000093510100B300000093520100B30000C2
:102DE0000093530100B300000093540100B30000AE
:102DF0000093550100B300000093560100B300009A
:102E00000093570100B300000093580100B3000085
:102E10000093590100B3000000935A0100B3000071
:102E200000935B0100B3000000935C0100B300005D
:102E300000935D0100B3000000935E0100B3000049
:102E400000935F0100B300000093600100B3000035
:102E50000093610100B300000093620100B3000021
:102E60000093630100B300000093640100B300000D
:102E70000093650100B300000093660100B30000F9
:102E80000093670100B300000093680100B30000E5
:102E90000093690100B3000000936A0100B30000D1
:102EA00000936B0100B3000000936C0100B30000BD
:102EB00000936D0100B3000000936E0100B30000A9
:102EC00000936F0100B300000093700100B3000095
:102ED0000093710100B300000093720100B3000081
:102EE0000093730100B300000093740100B300006D
:102EF0000093750100B300000093760100B3000059
:102F00000093770100B300000093780100B3000044
:102F10000093790100B3000000937A0100B3000030
:102F200000937B0100B3000000937C0100B300001C
:102F300000937D0100B3000000937E0100B3000008
:102F400000937F0100B300000093800100B30000F4
:102F50000093810100B300000093820100B30000E0
:102F60000093830100B300000093840100B30000CC
:102F70000093850100B300000093860100B30000B8
:102F80000093870100B300000093880100B30000A4
:102F90000093890100B3000000938A0100B3000090
:102FA00000938B0100B3000000938C0100B300007C
:102FB00000938D0100B3000000938E0100B3000068
:102FC00000938F0100B300000093900100B3000054
:102FD0000093910100B300000093920100B3000040
:102FE0000093930100B300000093940100B300002C
:102FF0000093950100B300000093960100B3000018
:103000000093970100B300000093980100B3000003
:103010000093990100B3000000939A0100B30000EF
:1030200000939B0100B3000000939C0100B30000DB
:1030300000939D0100B3000000939E0100B30000C7
:1030400000939F0100B300000093A00100B30000B3
:103050000093A10100B300000093A20100B300009F
:103060000093A30100B300000093A40100B300008B
:103070000093A50100B300000093A60100B3000077
:103080000093A70100B300000093A80100B3000063
:103090000093A90100B300000093AA0100B300004F
:1030A0000093AB0100B300000093AC0100B300003B
:1030B0000093AD0100B300000093AE0100B3000027
:1030C0000093AF0100B300000093B00100B3000013
:1030D0000093B10100B300000093B20100B30000FF
:1030E0000093B30100B300000093B40100B30000EB
:1030F0000093B50100B300000093B60100B30000D7
:103100000093B70100B300000093B80100B30000C2
:103110000093B90100B300000093BA0100B30000AE
:103120000093BB0100B300000093BC0100B300009A
:103130000093BD0100B300000093BE0100B3000086
:103140000093BF0100B300000093C00100B3000072
:103150000093C10100B300000093C20100B300005E
:103160000093C30100B300000093C40100B300004A
:103170000093C50100B300000093C60100B3000036
:103180000093C70100B300000093C80100B3000022
:103190000093C90100B300000093CA0100B300000E
:1031A0000093CB0100B300000093CC0100B30000FA
:1031B0000093CD0100B300000093CE0100B30000E6
:1031C0000093CF0100B300000093D00100B30000D2
:1031D0000093D10100B300000093D20100B30000BE
:1031E0000093D30100B300000093D40100B30000AA
:1031F0000093D50100B300000093D60100B3000096
:103200000093D70100B300000093D80100B3000081
:103210000093D90100B300000093DA0100B300006D
:103220000093DB0100B300000093DC0100B3000059
:103230000093DD0100B300000093DE0100B3000045
:103240000093DF0100B300000093E00100B3000031
:103250000093E10100B300000093E20100B300001D
:103260000093E30100B300000093E40100B3000009
:103270000093E50100B300000093E60100B30000F5
:103280000093E70100B300000093E80100B30000E1
:103290000093E90100B300000093EA0100B30000CD
:1032A0000093EB0100B300000093EC0100B30000B9
:1032B0000093ED0100B300000093EE0100B30000A5
:1032C0000093EF0100B300000093F00100B3000091
:1032D0000093F10100B300000093F20100B300007D
:1032E0000093F30100B300000093F40100B3000069
:1032F0000093F50100B300000093F60100B3000055
:103300000093F70100B300000093F80100B3000040
:103310000093F90100B300000093FA0100B300002C
:103320000093FB0100B300000093FC0100B3000018
:103330000093FD0100B300000093FE0100B3000004
:103340000093FF0100B300000093000200B30000EF
:103350000093010200B300000093020200B30000DA
:103360000093030200B300000093040200B30000C6
:103370000093050200B300000093060200B30000B2
:103380000093070200B300000093080200B300009E
:103390000093090200B3000000930A0200B300008A
:1033A00000930B0200B3000000930C0200B3000076
:1033B00000930D0200B3000000930E0200B3000062
:1033C00000930F0200B300000093100200B300004E
:1033D0000093110200B300000093120200B300003A
:1033E0000093130200B300000093140200B3000026
:1033F0000093150200B300000093160200B3000012
:103400000093170200B300000093180200B30000FD
:103410000093190200B3000000931A0200B30000E9
:1034200000931B0200B3000000931C0200B30000D5
:1034300000931D0200B3000000931E0200B30000C1
:1034400000931F0200B300000093200200B30000AD
:103450000093210200B300000093220200B3000099
:103460000093230200B300000093240200B3000085
:103470000093250200B300000093260200B3000071
:103480000093270200B300000093280200B300005D
:103490000093290200B3000000932A0200B3000049
:1034A00000932B0200B3000000932C0200B3000035
:1034B00000932D0200B3000000932E0200B3000021
:1034C00000932F0200B300000093300200B300000D
:1034D0000093310200B300000093320200B30000F9
:1034E0000093330200B300000093340200B30000E5
:1034F0000093350200B300000093360200B30000D1
:103500000093370200B300000093380200B30000BC
:103510000093390200B3000000933A0200B30000A8
:1035200000933B0200B3000000933C0200B3000094
:1035300000933D0200B3000000933E0200B3000080
:1035400000933F0200B300000093400200B300006C
:103550000093410200B300000093420200B3000058
:103560000093430200B300000093440200B3000044
:103570000093450200B300000093460200B3000030
:103580000093470200B300000093480200B300001C
:103590000093490200B3000000934A0200B3000008
:1035A00000934B0200B3000000934C0200B30000F4
:1035B00000934D0200B3000000934E0200B30000E0
:1035C00000934F0200B300000093500200B30000CC
:1035D0000093510200B300000093520200B30000B8
:1035E0000093530200B300000093540200B30000A4
:1035F0000093550200B300000093560200B3000090
:103600000093570200B300000093580200B300007B
:103610000093590200B3000000935A0200B3000067
:1036200000935B0200B3000000935C0200B3000053
:1036300000935D0200B3000000935E0200B300003F
:1036400000935F0200B300000093600200B300002B
:103650000093610200B300000093620200B3000017
:103660000093630200B300000093640200B3000003
:103670000093650200B300000093660200B30000EF
:103680000093670200B300000093680200B30000DB
:103690000093690200B3000000936A0200B30000C7
:1036A00000936B0200B3000000936C0200B30000B3
:1036B00000936D0200B3000000936E0200B300009F
:1036C00000936F0200B300000093700200B300008B
:1036D0000093710200B300000093720200B3000077
:1036E0000093730200B300000093740200B3000063
:1036F0000093750200B300000093760200B300004F
:103700000093770200B300000093780200B300003A
:103710000093790200B3000000937A0200B3000026
:1037200000937B0200B3000000937C0200B3000012
:1037300000937D0200B3000000937E0200B30000FE
:1037400000937F0200B300000093800200B30000EA
:103750000093810200B300000093820200B30000D6
:103760000093830200B300000093840200B30000C2
:103770000093850200B300000093860200B30000AE
:103780000093870200B300000093880200B300009A
:103790000093890200B3000000938A0200B3000086
:1037A00000938B0200B3000000938C0200B3000072
:1037B00000938D0200B3000000938E0200B300005E
:1037C00000938F0200B300000093900200B300004A
:1037D0000093910200B300000093920200B3000036
:1037E0000093930200B300000093940200B3000022
:1037F0000093950200B300000093960200B300000E
:103800000093970200B300000093980200B30000F9
:103810000093990200B3000000939A0200B30000E5
:1038200000939B0200B3000000939C0200B30000D1
:1038300000939D0200B3000000939E0200B30000BD
:1038400000939F0200B300000093A00200B30000A9
:103850000093A10200B300000093A20200B3000095
:103860000093A30200B300000093A40200B3000081
:103870000093A50200B300000093A60200B300006D
:103880000093A70200B300000093A80200B3000059
:103890000093A90200B300000093AA0200B3000045
:1038A0000093AB0200B300000093AC0200B3000031
:1038B0000093AD0200B300000093AE0200B300001D
:1038C0000093AF0200B300000093B00200B3000009
:1038D0000093B10200B300000093B20200B30000F5
:1038E0000093B30200B300000093B40200B30000E1
:1038F0000093B50200B300000093B60200B30000CD
:103900000093B70200B300000093B80200B30000B8
:103910000093B90200B300000093BA0200B30000A4
:103920000093BB0200B300000093BC0200B3000090
:103930000093BD0200B300000093BE0200B300007C
:103940000093BF0200B300000093C00200B3000068
:103950000093C10200B300000093C20200B3000054
:103960000093C30200B300000093C40200B3000040
:103970000093C50200B300000093C60200B300002C
:103980000093C70200B300000093C80200B3000018
:103990000093C90200B300000093CA0200B3000004
:1039A0000093CB0200B300000093CC0200B30000F0
:1039B0000093CD0200B300000093CE0200B30000DC
:1039C0000093CF0200B300000093D00200B30000C8
:1039D0000093D10200B300000093D20200B30000B4
:1039E0000093D30200B300000093D40200B30000A0
:1039F0000093D50200B300000093D60200B300008C
:103A00000093D70200B300000093D80200B3000077
:103A10000093D90200B300000093DA0200B3000063
:103A20000093DB0200B300000093DC0200B300004F
:103A30000093DD0200B300000093DE0200B300003B
:103A40000093DF0200B300000093E00200B3000027
:103A50000093E10200B300000093E20200B3000013
:103A60000093E30200B300000093E40200B30000FF
:103A70000093E50200B300000093E60200B30000EB
:103A80000093E70200B300000093E80200B30000D7
:103A90000093E90200B300000093EA0200B30000C3
:103AA0000093EB0200B300000093EC0200B30000AF
:103AB0000093ED0200B300000093EE0200B300009B
:103AC0000093EF0200B300000093F00200B3000087
:103AD0000093F10200B300000093F20200B3000073
:103AE0000093F3020093F40200B300000093F50288
:103AF00000B300000093F60200B300000093F70249
:103B000000B300000093F80200B300000093F90234
:103B100000B300000093FA0200B300000093FB0220
:103B200000B300000093FC0200B300000093FD020C
:103B300000B300000093FE0200B300000093FF02F8
:103B400000B300000093000300B3000000930103E2
:103B500000B300000093020300B3000000930303CE
:103B600000B300000093040300B3000000930503BA
:103B700000B300000093060300B3000000930703A6
:103B800000B300000093080300B300000093090392
:103B900000B3000000930A0300B3000000930B037E
:103BA00000B3000000930C0300B3000000930D036A
:103BB00000B3000000930E0300B3000000930F0356
:103BC00000B300000093100300B300000093110342
:103BD00000B300000093120300B30000009313032E
:103BE00000B300000093140300B30000009315031A
:103BF00000B300000093160300B300000093170306
:103C000000B300000093180300B3000000931903F1
:103C100000B3000000931A0300B3000000931B03DD
:103C200000B3000000931C0300B3000000931D03C9
:103C300000B3000000931E0300B3000000931F03B5
:103C400000B300000093200300B3000000932103A1
:103C500000B300000093220300B30000009323038D
:103C600000B300000093240300B300000093250379
:103C700000B300000093260300B300000093270365
:103C800000B300000093280300B300000093290351
:103C900000B3000000932A0300B3000000932B033D
:103CA00000B3000000932C0300B3000000932D0329
:103CB00000B3000000932E0300B3000000932F0315
:103CC00000B300000093300300B300000093310301
:103CD00000B300000093320300B3000000933303ED
:103CE00000B300000093340300B3000000933503D9
:103CF00000B300000093360300B3000000933703C5
:103D000000B300000093380300B3000000933903B0
:103D100000B3000000933A0300B3000000933B039C
:103D200000B3000000933C0300B3000000933D0388
:103D300000B3000000933E0300B3000000933F0374
:103D400000B300000093400300B300000093410360
:103D500000B300000093420300B30000009343034C
:103D600000B300000093440300B300000093450338
:103D700000B300000093460300B300000093470324
:103D800000B300000093480300B300000093490310
:103D900000B3000000934A0300B3000000934B03FC
:103DA00000B3000000934C0300B3000000934D03E8
:103DB00000B3000000934E0300B3000000934F03D4
:103DC00000B300000093500300B3000000935103C0
:103DD00000B300000093520300B3000000935303AC
:103DE00000B300000093540300B300000093550398
:103DF00000B300000093560300B300000093570384
:103E00000093580300B300000093590300B300006F
:103E100000935A0300B3000000935B0300B300005B
:103E200000935C0300B3000000935D0300B3000047
:103E300000935E0300B3000000935F0300B3000033
:103E40000093600300B300000093610300B300001F
:103E50000093620300B300000093630300B300000B
:103E60000093640300B300000093650300B30000F7
:103E70000093660300B300000093670300B30000E3
:103E80000093680300B300000093690300B30000CF
:103E900000936A0300B3000000936B0300B30000BB
:103EA00000936C0300B3000000936D0300B30000A7
:103EB00000936E0300B3000000936F0300B3000093
:103EC0000093700300B300000093710300B300007F
:103ED0000093720300B300000093730300B300006B
:103EE0000093740300B300000093750300B3000057
:103EF0000093760300B300000093770300B3000043
:103F00000093780300B300000093790300B300002E
:103F100000937A0300B3000000937B0300B300001A
:103F200000937C0300B3000000937D0300B3000006
:103F300000937E0300B3000000937F0300B30000F2
:103F40000093800300B300000093810300B30000DE
:103F50000093820300B300000093830300B30000CA
:103F60000093840300B300000093850300B30000B6
:103F70000093860300B300000093870300B30000A2
:103F80000093880300B300000093890300B300008E
:103F900000938A0300B3000000938B0300B300007A
:103FA00000938C0300B3000000938D0300B3000066
:103FB00000938E0300B3000000938F0300B3000052
:103FC0000093900300B300000093910300B300003E
:103FD0000093920300B300000093930300B300002A
:103FE0000093940300B300000093950300B3000016
:103FF0000093960300B300000093970300B3000002
:104000000093980300B300000093990300B30000ED
:1040100000939A0300B3000000939B0300B30000D9
:1040200000939C0300B3000000939D0300B30000C5
:1040300000939E0300B3000000939F0300B30000B1
:104040000093A00300B300000093A10300B300009D
:104050000093A20300B300000093A30300B3000089
:104060000093A40300B300000093A50300B3000075
:104070000093A60300B300000093A70300B3000061
:104080000093A80300B300000093A90300B300004D
:104090000093AA0300B300000093AB0300B3000039
:1040A0000093AC0300B300000093AD0300B3000025
:1040B0000093AE0300B300000093AF0300B3000011
:1040C0000093B00300B300000093B10300B30000FD
:1040D0000093B20300B300000093B30300B30000E9
:1040E0000093B40300B300000093B50300B30000D5
:1040F0000093B60300B300000093B70300B30000C1
:104100000093B80300B300000093B90300B30000AC
:104110000093BA0300B300000093BB030093BC03F9
:1041200000B300000093BD0300B300000093BE0382
:1041300000B300000093BF0300B300000093C0036E
:1041400000B300000093C10300B300000093C2035A
:1041500000B300000093C30300B300000093C40346
:1041600000B300000093C50300B300000093C60332
:1041700000B300000093C70300B300000093C8031E
:1041800000B300000093C90300B300000093CA030A
:1041900000B300000093CB0300B300000093CC03F6
:1041A00000B300000093CD0300B300000093CE03E2
:1041B00000B300000093CF0300B300000093D003CE
:1041C00000B300000093D10300B300000093D203BA
:1041D00000B300000093D30300B300000093D403A6
:1041E00000B300000093D50300B300000093D60392
:1041F00000B300000093D70300B300000093D8037E
:1042000000B300000093D90300B300000093DA0369
:1042100000B300000093DB0300B300000093DC0355
:1042200000B300000093DD0300B300000093DE0341
:1042300000B300000093DF0300B300000093E0032D
:1042400000B300000093E10300B300000093E20319
:1042500000B300000093E30300B300000093E40305
:1042600000B300000093E50300B300000093E603F1
:1042700000B300000093E70300B300000093E803DD
:1042800000B300000093E90300B300000093EA03C9
:1042900000B300000093EB0300B300000093EC03B5
:1042A00000B300000093ED0300B300000093EE03A1
:1042B00000B300000093EF0300B300000093F0038D
:1042C00000B300000093F10300B300000093F20379
:1042D00000B300000093F30300B300000093F40365
:1042E00000B300000093F50300B300000093F60351
:1042F00000B300000093F70300B300000093F8033D
:1043000000B300000093F90300B300000093FA0328
:1043100000B300000093FB0300B300000093FC0314
:1043200000B300000093FD0300B300000093FE0300
:1043300000B300000093FF0300B3000000930004EB
:1043400000B300000093010400B3000000930204D6
:1043500000B300000093030400B3000000930404C2
:1043600000B300000093050400B3000000930604AE
:1043700000B300000093070400B30000009308049A
:1043800000B300000093090400B3000000930A0486
:1043900000B3000000930B0400B3000000930C0472
:1043A00000B3000000930D0400B3000000930E045E
:1043B00000B3000000930F0400B30000009310044A
:1043C00000B300000093110400B300000093120436
:1043D00000B300000093130400B300000093140422
:1043E00000B300000093150400B30000009316040E
:1043F00000B300000093170400B3000000931804FA
:1044000000B300000093190400B3000000931A04E5
:1044100000B3000000931B0400B3000000931C04D1
:1044200000B3000000931D0400B3000000931E04BD
:1044300000B3000000931F040093200400B30000A9
:104440000093210400B300000093220400B3000095
:104450000093230400B300000093240400B3000081
:104460000093250400B300000093260400B300006D
:104470000093270400B300000093280400B3000059
:104480000093290400B3000000932A0400B3000045
:1044900000932B0400B3000000932C0400B3000031
:1044A00000932D0400B3000000932E0400B300001D
:1044B00000932F0400B300000093300400B3000009
:1044C0000093310400B300000093320400B30000F5
:1044D0000093330400B300000093340400B30000E1
:1044E0000093350400B300000093360400B30000CD
:1044F0000093370400B300000093380400B30000B9
:104500000093390400B3000000933A0400B30000A4
:1045100000933B0400B3000000933C0400B3000090
:1045200000933D0400B3000000933E0400B300007C
:1045300000933F0400B300000093400400B3000068
:104540000093410400B300000093420400B3000054
:104550000093430400B300000093440400B3000040
:104560000093450400B300000093460400B300002C
:104570000093470400B300000093480400B3000018
:104580000093490400B3000000934A0400B3000004
:1045900000934B0400B3000000934C0400B30000F0
:1045A00000934D0400B3000000934E0400B30000DC
:1045B00000934F0400B300000093500400B30000C8
:1045C0000093510400B300000093520400B30000B4
:1045D0000093530400B300000093540400B30000A0
:1045E0000093550400B300000093560400B300008C
:1045F0000093570400B300000093580400B3000078
:104600000093590400B3000000935A0400B3000063
:1046100000935B0400B3000000935C0400B300004F
:1046200000935D0400B3000000935E0400B300003B
:1046300000935F0400B300000093600400B3000027
:104640000093610400B300000093620400B3000013
:104650000093630400B300000093640400B30000FF
:104660000093650400B300000093660400B30000EB
:104670000093670400B300000093680400B30000D7
:104680000093690400B3000000936A0400B30000C3
:1046900000936B0400B3000000936C0400B30000AF
:1046A00000936D0400B3000000936E0400B300009B
:1046B00000936F0400B300000093700400B3000087
:1046C0000093710400B300000093720400B3000073
:1046D0000093730400B300000093740400B300005F
:1046E0000093750400B300000093760400B300004B
:1046F0000093770400B300000093780400B3000037
:104700000093790400B3000000937A0400B3000022
:1047100000937B0400B3000000937C0400B300000E
:1047200000937D0400B3000000937E0400B30000FA
:1047300000937F0400B300000093800400B30000E6
:104740000093810400B300000093820400B30000D2
:10475000009383040093840400B300000093850455
:1047600000B300000093860400B3000000938704A8
:1047700000B300000093880400B300000093890494
:1047800000B3000000938A0400B3000000938B0480
:1047900000B3000000938C0400B3000000938D046C
:1047A00000B3000000938E0400B3000000938F0458
:1047B00000B300000093900400B300000093910444
:1047C00000B300000093920400B300000093930430
:1047D00000B300000093940400B30000009395041C
:1047E00000B300000093960400B300000093970408
:1047F00000B300000093980400B3000000939904F4
:1048000000B3000000939A0400B3000000939B04DF
:1048100000B3000000939C0400B3000000939D04CB
:1048200000B3000000939E0400B3000000939F04B7
:1048300000B300000093A00400B300000093A104A3
:1048400000B300000093A20400B300000093A3048F
:1048500000B300000093A40400B300000093A5047B
:1048600000B300000093A60400B300000093A70467
:1048700000B300000093A80400B300000093A90453
:1048800000B300000093AA0400B300000093AB043F
:1048900000B300000093AC0400B300000093AD042B
:1048A00000B300000093AE0400B300000093AF0417
:1048B00000B300000093B00400B300000093B10403
:1048C00000B300000093B20400B300000093B304EF
:1048D00000B300000093B40400B300000093B504DB
:1048E00000B300000093B60400B300000093B704C7
:1048F00000B300000093B80400B300000093B904B3
:1049000000B300000093BA0400B300000093BB049E
:1049100000B300000093BC0400B300000093BD048A
:1049200000B300000093BE0400B300000093BF0476
:1049300000B300000093C00400B300000093C10462
:1049400000B300000093C20400B300000093C3044E
:1049500000B300000093C40400B300000093C5043A
:1049600000B300000093C60400B300000093C70426
:1049700000B300000093C80400B300000093C90412
:1049800000B300000093CA0400B300000093CB04FE
:1049900000B300000093CC0400B300000093CD04EA
:1049A00000B300000093CE0400B300000093CF04D6
:1049B00000B300000093D00400B300000093D104C2
:1049C00000B300000093D20400B300000093D304AE
:1049D00000B300000093D40400B300000093D5049A
:1049E00000B300000093D60400B300000093D70486
:1049F00000B300000093D80400B300000093D90472
:104A000000B300000093DA0400B300000093DB045D
:104A100000B300000093DC0400B300000093DD0449
:104A200000B300000093DE0400B300000093DF0435
:104A300000B300000093E00400B300000093E10421
:104A400000B300000093E20400B300000093E3040D
:104A500000B300000093E40400B300000093E504F9
:104A600000B300000093E60400B300000093E704E5
:104A70000093E80400B300000093E90400B30000D1
:104A80000093EA0400B300000093EB0400B30000BD
:104A90000093EC0400B300000093ED0400B30000A9
:104AA0000093EE0400B300000093EF0400B3000095
:104AB0000093F00400B300000093F10400B3000081
:104AC0000093F20400B300000093F30400B300006D
:104AD0000093F40400B300000093F50400B3000059
:104AE0000093F60400B300000093F70400B3000045
:104AF0000093F80400B300000093F90400B3000031
:104B00000093FA0400B300000093FB0400B300001C
:104B10000093FC0400B300000093FD0400B3000008
:104B20000093FE0400B300000093FF0400B30000F4
:104B3000089508954091770000B3041718F011F01C
:104B40000C94A4250C94BF25A6E6B0E00D911C9111
:104B50000F5F1F4FA6E6B0E00D931C93A6E6B0E0F2
:104B60000D911C91083E53E0150718F011F00C94BC
:104B7000BB250C94BD250C94BF250C949A25AF93AE
:104B8000BF93B1E0A0E00000000080B38D93B5308A
:104B9000D0F38F919F91BF91AF910895409177008D
:104BA00000B3041718F011F00C94D8250C94F325D9
:104BB000A6E6B0E00D911C910F5F1F4FA6E6B0E096
:104BC0000D931C93A6E6B0E00D911C91083E53E0B6
:104BD000150718F011F00C94EF250C94F1250C94A6
:104BE000F3250C94CE25AF93BF93B1E0A0E0000075
:104BF00000000000000000000000000000000000B5
:104C00000000000000000000000080B38D93B5306C
:104C100070F38F919F91BF91AF910895409177006C
:104C200000B3041718F011F00C9418260C943326D6
:104C3000A6E6B0E00D911C910F5F1F4FA6E6B0E015
:104C40000D931C93A6E6B0E00D911C91083E53E035
:104C5000150718F011F00C942F260C9431260C94A3
:104C600033260C940E26AF93BF93B1E0A0E00BE087
:104C70000A95F1F7000080B38D93B530C0F38F91A2
:104C80009F91BF91AF9108954091770000B30417B1
:104C900018F011F00C944E260C946926A6E6B0E0AC
:104CA0000D911C910F5F1F4FA6E6B0E00D931C9372
:104CB000A6E6B0E00D911C91083E53E0150718F0F0
:104CC00011F00C9465260C9467260C9469260C94BC
:104CD0004426AF93BF93B1E0A0E008E10A95F1F755
:104CE0000000000080B38D93B530B8F38F919F9191
:104CF000BF91AF9108954091770000B3041718F069
:104D000011F00C9485260C94A026A6E6B0E00D9137
:104D10001C910F5F1F4FA6E6B0E00D931C93A6E613
:104D2000B0E00D911C91083E53E0150718F011F00A
:104D30000C949C260C949E260C94A0260C947B2606
:104D4000AF93BF93B1E0A0E000E40A95F1F7000053
:104D5000000080B38D93B530B8F38F919F91BF91D0
:104D6000AF9108954091770000B3041718F011F047
:104D70000C94BC260C94D726A6E6B0E00D911C91AD
:104D80000F5F1F4FA6E6B0E00D931C93A6E6B0E0C0
:104D90000D911C91083E53E0150718F011F00C948A
:104DA000D3260C94D5260C94D7260C94B226AF9318
:104DB000BF93B1E0A0E003E80A95F1F7000080B3EB
:104DC0008D93B530C0F38F919F91BF91AF910895AE
:104DD0004091770000B3041718F011F00C94F226FC
:104DE0000C940D27A6E6B0E00D911C910F5F1F4FAC
:104DF000A6E6B0E00D931C93A6E6B0E00D911C91E1
:104E0000083E53E0150718F011F00C9409270C9494
:104E10000B270C940D270C94E826AF93BF93B1E0B9
:104E2000A0E00FEF0A95F1F70FEF0A95F1F70AE905
:104E30000A95F1F7000080B38D93B53090F38F9110
:104E40009F91BF91AF910895A881B9818C91809372
:104E50006400C39A82E390E00E943F2DC39882E3EE
:104E600090E00E943F2DC39AC19A82E390E00E9495
:104E70003F2D81E1D2018C9381E00E94552D0E944B
:104E8000212C229681E00E94512D84E190E00E9425
:104E90003F2D80EDD2018C9381E00E94552D0E9420
:104EA000212C229681E00E94512D87E0D2018C9323
:104EB00081E00E94552D0E942B2C229681E00E94B9
:104EC000512D82E4D2018C9381E00E94552D0E94E5
:104ED0002B2C229681E00E94512D88E1D2018C93E7
:104EE00081E00E94552D0E942B2C229681E00E9489
:104EF000512D81EDD2018C9381E00E94552D0E94AD
:104F0000212C229681E00E94512D80E0D2018C93C9
:104F100081E00E94552D0E942B2C229681E00E9458
:104F2000512D87E0D2018C9381E00E94552D0E9483
:104F30002B2C229681E00E94512D80E1D2018C938E
:104F400081E00E94552D0E942B2C229681E00E9428
:104F5000512D82EDD2018C9381E00E94552D0E944B
:104F6000212C229681E00E94512D81E0D2018C9368
:104F700081E00E94552D0E942B2C229681E00E94F8
:104F8000512D82E0D2018C9381E00E94552D0E9428
:104F90002B2C229681E00E94512D80ECD2018C9323
:104FA00081E00E94552D0E94212C229681E00E94D2
:104FB000512D80E1D2018C9381E00E94552D0E94F9
:104FC0002B2C229681E00E94512D8BE3D2018C93F1
:104FD00081E00E94552D0E942B2C229681E00E9498
:104FE000512D80E0D2018C9381E00E94552D0E94CA
:104FF0002B2C229681E00E94512D82E0D2018C93CD
:1050000081E00E94552D0E942B2C229681E00E9467
:10501000512D81E1D2018C9381E00E94552D0E9497
:105020002B2C229681E00E94512D85ECD2018C938D
:1050300081E00E94552D0E94212C229681E00E9441
:10504000512D83E0D2018C9381E00E94552D0E9466
:105050002B2C229681E00E94512D88ECD2018C935A
:1050600081E00E94552D0E94212C229681E00E9411
:10507000512D80E0D2018C9381E00E94552D0E9439
:105080002B2C229681E00E94512D82E3D2018C9339
:1050900081E00E94552D0E942B2C229681E00E94D7
:1050A000512D86E3D2018C9381E00E94552D0E9400
:1050B0002B2C229681E00E94512D85E4D2018C9305
:1050C00081E00E94552D0E942B2C229681E00E94A7
:1050D000512D86E0D2018C9381E00E94552D0E94D3
:1050E0002B2C229681E00E94512D86E1D2018C93D7
:1050F00081E00E94552D0E942B2C229681E00E9477
:10510000512D87E3D2018C9381E00E94552D0E949E
:105110002B2C229681E00E94512D85E7D2018C93A1
:1051200081E00E94552D0E942B2C229681E00E9446
:10513000512D87E7D2018C9381E00E94552D0E946A
:105140002B2C229681E00E94512D84E5D2018C9374
:1051500081E00E94552D0E942B2C229681E00E9416
:10516000512D8CE0D2018C9381E00E94552D0E943C
:105170002B2C229681E00E94512D80E0D2018C934D
:1051800081E00E94552D0E942B2C229681E00E94E6
:10519000512D86E3D2018C9381E00E94552D0E940F
:1051A000212C229681E00E94512D8AE0D2018C931D
:1051B00081E00E94552D0E942B2C229681E00E94B6
:1051C000512D8AE3D2018C9381E00E94552D0E94DB
:1051D000212C229681E00E94512D85E5D2018C93ED
:1051E00081E00E94552D0E942B2C229681E00E9486
:1051F000512D8AE2D2018C9381E00E94552D0E94AC
:10520000212C229681E00E94512D80E0D2018C93C6
:1052100081E00E94552D0E942B2C229681E00E9455
:10522000512D80E0D2018C9381E00E94552D0E9487
:105230002B2C229681E00E94512D81E0D2018C938B
:1052400081E00E94552D0E942B2C229681E00E9425
:10525000512D8FE3D2018C9381E00E94552D0E9445
:105260002B2C229681E00E94512D8BE2D2018C934F
:1052700081E00E94552D0E94212C229681E00E94FF
:10528000512D80E0D2018C9381E00E94552D0E9427
:105290002B2C229681E00E94512D80E0D2018C932C
:1052A00081E00E94552D0E942B2C229681E00E94C5
:1052B000512D81E0D2018C9381E00E94552D0E94F6
:1052C0002B2C229681E00E94512D80EED2018C93EE
:1052D00081E00E94552D0E942B2C229681E00E9495
:1052E000512D88E790E00E943F2D89E2D2018C93F6
:1052F00081E00E94552D0E94212C229681E00E947F
:10530000512D88E790E00E943F2D80EE91E0A0E6CD
:10531000B0E08D939C9380E491E0A2E6B0E08D93A1
:105320009C93089584E00E94552DD2010E94772D10
:1053300082E00E94552DD2010E94772D82E00E94CA
:10534000552D8FED91E0D2018D939C9382E00E94C8
:10535000552D8FE391E0D2018D939C9382E00E94C2
:10536000552D0E94352C289688E00E94512DC09A18
:10537000AA81BB8111968C9185BBAA81BB818C913E
:105380008BBBA881B9810E94792D4FEF57E562E070
:1053900070E0A881B9810D911D912D913C910E94E1
:1053A0007F2D1CF011F00C94DD29C198C19AA881C1
:1053B000B9810E94DB2C0C94C52984E0481A80E056
:1053C000580A2296089582E00E94552D82E00E949C
:1053D000552D82E00E94552D81E00E94552D81E0DF
:1053E0000E94552D81E00E94552D81E00E94552D8F
:1053F00081E00E94552D81E00E94552D81E00E94A0
:10540000552D81E00E94552D81E00E94552D81E0AF
:105410000E94552D81E00E94552D81E00E94552D5E
:1054200082E00E94552D82E00E94552D82E00E946C
:10543000552D81E00E94552DA8A9B9A90E94AB2D38
:10544000082F41E0041BA885B9850C9380E0AA8D44
:10545000BB8D8C93A885B9854C91AA8DBB8D0C9181
:10546000041718F011F00C94E02BAAA5BBA50C9121
:10547000013011F00C94402AE8EFFDE10E94D52C98
:10548000AAA5BBA50C91023011F00C944B2AECEEAE
:10549000F0E20E94D52CAAA5BBA50C91033011F017
:1054A0000C94562AECEEF0E20E94D52CAA8DBB8D0E
:1054B0000D9111270F5F1F4FAAA1BBA10D931C9344
:1054C000AAA1BBA18C91E8A9F9A901E00A93ADA119
:1054D000BEA10E948C2D0E94D82CAE89BF890E944B
:1054E000732D0C920E94D52C0E94D82CAC89BD89BA
:1054F0000E94732D0C920E94D52C0E94D82CAA8950
:10550000BB890E94732D0C920E94D52C0E94D82C2E
:10551000A889B9890E94732D0C920E94D52CACA148
:10552000BDA18C91082F112700521040AAA1BBA148
:105530000D931C9381E0A88DB98D8C93AAA1BBA17A
:105540004D915C91A88DB98D0D9111270417150708
:1055500018F011F00C94D42A81E0AC8DBD8D8C93A1
:10556000AA89BB894C91AC8DBD8D0C91041718F0A4
:1055700011F00C94CC2A0E94D82CAE8DBF8D0E94C5
:10558000732D0C920E94D52CAC8DBD8D8C918F5FAC
:105590008C9310F40C94B02AA88DB98D8C918F5FE8
:1055A0008C9310F40C949E2AAA89BB890C91AE8925
:1055B000BF894C910E949B2DAE85BF850C93AE890F
:1055C000BF890C9148E0049F0C92AE89BF898C91F1
:1055D00081508C93AE85BF858C9181508C9380E0F7
:1055E000AA85BB858C93AE89BF894C91AA85BB8562
:1055F0000C91041718F011F00C94D82BAA85BB85D8
:105600000D911127ACA5BDA54D915C91040F151FFF
:10561000A8A1B9A10D931C9380E0AC85BD858C93A6
:10562000AE85BF854C91AC85BD850C91041718F0F3
:1056300011F00C94D02B0E94D82CAE8DBF8D0E94FF
:10564000732D0C920E94D52CAC85BD858C91AE81BA
:10565000BF818D9388278C93AA8DBB8D0D911127C7
:10566000AC89BD894D9155270E945B2DAAA1BBA194
:105670000D931C93AE81BF810D911C91AAA1BBA17A
:105680004D915C91040F151FAE81BF810D931C934A
:10569000AE81BF810D911C91AEA5BFA54D915C91CE
:1056A000040F151FAE81BF810D931C9380E0A8816C
:1056B000B9818C93A881B9810C91073018F011F051
:1056C0000C94C82BA8A1B9A10D911C91A881B981F6
:1056D0004D915527040F151FAC81BD810D931C936F
:1056E000AE8DBF8D8C9180FBAA81BB81882780F90C
:1056F0008D9388278C93AA81BB810D911C910130D9
:1057000050E0150711F00C948F2BA8A5B9A58D9129
:105710009C91AA81BB818D939C930C94972BAEA1F5
:10572000BFA18D919C91AA81BB818D939C93AE81E9
:10573000BF818D919C91D2018D939C9382E00E94B8
:10574000552DAE81BF818D919C91D2018D939C93FB
:1057500082E00E94552DAE81BF818D919C91D20136
:105760008D939C9382E00E94552D0E94E62B2696F5
:1057700086E00E94512D91E0AE8DBF8D0E946B2D71
:10578000A881B9818C918F5F8C9310F40C945A2B63
:10579000AC85BD858C918F5F8C9310F40C94102B8D
:1057A000AA85BB858C91885F8C9310F40C94F32AA6
:1057B000AA8DBB8D8C918F5F8C9310F40C942A2A48
:1057C00089E1481A80E0580AA6960895AC81BD8107
:1057D0008D919C91D2018D939C9382E00E94552DD6
:1057E000AC81BD818D919C91D2018D939C9382E07F
:1057F0000E94552DA885B9858D919C91D2018D93DC
:105800009C9382E00E94552DA885B9858D919C912D
:10581000D2018D939C9382E00E94552D0E94352CDD
:10582000289688E00E94512DC09AA881B9811196CE
:105830008C9185BBA881B9818C918BBBC198C19A91
:105840000895C09870E075BBA881B9818C918BBB1D
:10585000C198C19A0895C09A70E075BBA881B981BA
:105860008C918BBBC198C19A089582E00E94552DFE
:10587000A885B9858D919C91A881B9818D939C93C0
:10588000AE81BF818D919C91A885B9858D939C93A4
:105890000FED11E0A881B9814D915C91041B150BAE
:1058A000AE81BF810D931C93AC81BD818D919C9184
:1058B000A881B9818D939C93AA81BB818D919C9184
:1058C000AC81BD818D939C930FED11E0A881B981CE
:1058D0004D915C91041B150BAA81BB810D931C9308
:1058E000AE81BF818D919C91A881B9818D939C934C
:1058F000AA81BB818D919C91AE81BF818D939C9338
:10590000A881B9818D919C91AA81BB818D939C9333
:1059100070E075BBC098AAE2ABBBC198C19AC09AAF
:10592000A885B98511968C918BBBC198C19AA88521
:10593000B9858C918BBBC198C19AAC81BD81119600
:105940008C918BBBC198C19AAC81BD818C918BBB72
:10595000C198C19AC098ABE2ABBBC198C19AC09A3A
:10596000AE81BF8111968C918BBBC198C19AAE81DB
:10597000BF818C918BBBC198C19AAA81BB811196C2
:105980008C918BBBC198C19AAA81BB818C918BBB36
:10599000C198C19AC098ACE2ABBBC198C19A82E0F1
:1059A000481A80E0580A229608958E2E9F2E089558
:1059B000E82DF92D08950D911D912D913C910F5FCA
:1059C0001F4F2F4F3F4F3C932E931E930E930895DE
:1059D000ED91FC91EF5FFF4FFC93EE930895ED91F5
:1059E000FC91E150F040FC93EE93089509D00E94A1
:1059F0005B2D00FC10D0089503D01ED001F8F9CF24
:105A00000024E89457FF02C009D0689400F80BD036
:105A100010F80124089502D009D0089550954095BA
:105A20004F5F5F4F0895E89417FF08950095109514
:105A30000F5F1F4F68940895352F242FE894452B4E
:105A400011F468940895512F402F0027112780E109
:105A5000440F551F001F111F021B130B416018F448
:105A6000020F131F4E7F8A9599F708953197F1F72A
:105A70000895689462F80895E89462F80895EF93A1
:105A8000FF93EE27E82BE92B31F0E0EAFFE03197B6
:105A9000F1F70197D1F7FF91EF910895481A590A4C
:105AA0000895481A8827580A089599275A924A92C1
:105AB000480E591E08950F92B801469F8001479FD6
:105AC000100D569F100D0F9008950E94732D0D928A
:105AD0000020D9F70895903029F08C9186959A95F9
:105AE000E9F78C930895C89531960020089582E0D7
:105AF00001C084E099279D938A95E9F708950417DA
:105B0000150726073707089588278D9308958191F3
:105B10008D938823E1F7089509919191992351F08C
:105B20008A95D9F73197002329F081918D930A95B1
:105B30008823C9F7E9CFFF93881BF9E0001FFA9586
:105B400011F4FF910895881F841B18F4840F889422
:105B5000F5CF0894F3CF8FEF83959D919923E1F7CB
:105B60000895494C4939343831204E45572032394F
:105B70005F30395F323031375C30345F31305F3223
:105B80003031375F3030352E6261730020202020A5
:105B900020202020204F5343494C4C4F534B4F5013
:105BA000205620312E30312020202020202020207F
:105BB00020202020200031302056000035205620A3
:105BC0000000322056200000312056200000302EE8
:105BD00035560000302E32560000302E315600006F
:105BE00035306D5600002000322E352075730000D0
:105BF000352E302075730000313020757320000081
:105C0000323020757320000035302075732000007D
:105C1000302E31206D730000302E32206D73000065
:105C2000302E35206D73000031206D732020000070
:105C300035206D7320200000506175736520202091
:105C4000000041430000444300002020000053595D
:105C50004E430000312E30205600302E373556008E
:105C6000302E35205600302E32355600302E302062
:105C70005600302020322E352020203520202020B4
:105C8000372E3520203130202031322E3520203162
:105C900035202031372E3520203230202032322E50
:105CA0003520203235202032372E3520000030209C
:105CB0002030352020202031302020203135202078
:105CC0002032302020203235202020333020202068
:105CD000333520202034302020203435202020353A
:105CE0003020202035352020200030202020313069
:105CF000202020323020202033302020203430203B
:105D00002020353020202036302020203730202021
:105D100020383020202039302020313030202031F0
:105D2000313020200000302020203230202020344C
:105D300030202020363020202038302020313030D4
:105D400020203132302020313430202031363020B4
:105D500020313830202032303020203232302020A4
:105D600000003020202035302020313030202031FC
:105D70003530202032303020203235302020333072
:105D8000302020333530202034303020203435305E
:105D900020203530302020353530202000003020C4
:105DA00020302E312020302E322020302E33202063
:105DB000302E342020302E352020302E362020303A
:105DC0002E372020302E382020302E392020312E22
:105DD000302020312E3120200000302020302E3283
:105DE0002020302E342020302E362020302E382017
:105DF00020312E302020312E322020312E34202010
:105E0000312E362020312E382020322E30202032E4
:105E10002E3220200000302020302E352020312E40
:105E2000302020312E352020322E302020322E35C9
:105E30002020332E302020332E352020342E3020C9
:105E400020342E352020352E302020352E352020B0
:105E5000000030202020312020202032202020204F
:105E600033202020203420202020352020202036E0
:105E700020202020372020202038202020203920DA
:105E800020202031302020203131202000003020FF
:105E900020202035202020313020202031352020A6
:105EA0002032302020203235202020333020202086
:105EB0003335202020343020202034352020203558
:0A5EC000302020203535202000009E
:00000001FF
